S01700004763634170706C69636174696F6E352E7372656357
S11300000C9434000C9451000C9451000C94510045
S11300100C9451000C9451000C9451000C94510018
S11300200C9451000C9451000C9451000C94510008
S11300300C9451000C9451000C9451000C945100F8
S11300400C9451000C9451000C9451000C945100E8
S11300500C9451000C9451000C9451000C945100D8
S11300600C9451000C94510011241FBECFEFD8E022
S1130070DEBFCDBF11E0A0E0B1E0EEE2F6E002C0E9
S113008005900D92A034B107D9F721E0A0E4B1E0C6
S113009001C01D92A034B207E1F70E9453000C94F2
S11300A015030C940000CF93DF93CDB7DEB76097B0
S11300B00FB6F894DEBF0FBECDBF88B1897F88B973
S11300C087B1866087B9419A0E94AE022FE38DE022
S11300D093E0215080409040E1F700C000000E946E
S11300E0FD022FE38DE093E0215080409040E1F742
S11300F000C000000E94D8002FE38DE093E021505F
S113010080409040E1F700C0000087E30E94C800EF
S1130110823929F480E091E00E9499020CC0805950
S1130120823028F48FE091E00E94990204C08EE1AD
S113013091E00E94990282E00E94C800682F6062E8
S113014082E00E94BB0083E00E94C800682F6068C0
S113015083E00E94BB002FE78DE89BE5215080409F
S11301609040E1F700C00000BE016F5F7F4F82E561
S11301700E942D02F9CFCF93C62F2A98880F8E772D
S11301800E9406038C2F0E9406032A9ACF91089599
S11301902A98880F8E7780680E94060380E00E9468
S11301A006032A9A08956FE081E00E94BB00089537
S11301B00E94D3006DE88AE20E94BB006EE38BE2EA
S11301C00E94BB006EE18CE20E94BB0060E08DE205
S11301D00E94BB0060E485E10E94BB006DE381E105
S11301E00E94BB0084E10E94C800982F937029F4F8
S11301F0682F636084E10E94BB0008953F924F9290
S11302005F926F927F928F929F92AF92BF92CF92A2
S1130210DF92EF92FF920F931F93CF93DF93982E69
S1130220F62EE72E442E822E332E58018CE098169B
S113023009F4C9C0EEE09E1203C010E102E102C05D
S113024010E000E084E00E94C800682F6F7784E02B
S11302500E94BB008AE00E94C800682F60688AE0A0
S11302600E94BB0060E081E00E94BB00512C612C25
S1130270712C411451046104710419F415C010E384
S113028007E7CF2DDE2DC12CD12C7601699189E0B1
S11302900E94BB00FFEFCF1ADF0AEF0AFF0AC41463
S11302A0D504E604F70490F3692D81E00E94BB00B5
S11302B08CE0981208C08DE00E94C800682F606826
S11302C08DE00E94BB0084E00E94C800F82EC0E0CC
S11302D0D0E011600AC084E00E94C800F82E219684
S11302E0CF3CE7E0DE0709F48CC0812F8F2199F31E
S11302F092C00170F02211F0C2E001C0C1E0FCE044
S11303009F1298C08AE00E94C800482E8CE00E9488
S1130310C800282F2770A9F0842D90E00197880F3A
S1130320991F880F991F880F991F820F911D092EFD
S1130330000CAA0BBB0BF50180839183A283B383CA
S113034011C0842D90E0880F991F880F991F880F82
S1130350991F092E000CAA0BBB0BF5018083918316
S1130360A283B383442071F0842D813108F080E1AD
S1130370482E512C612C712C4114510461047104D8
S113038029F458C0412C512C32014394082D132DCB
S1130390C12CD12C760189E00E94C800F801819318
S11303A08F01FFEFCF1ADF0AEF0AFF0AC414D50446
S11303B0E604F70480F33EC06CE081E00E94BB00D9
S11303C010E307E778CF84E00E94C800682F6F77B6
S11303D084E00E94BB008AE00E94C800682F606825
S11303E08AE00E94BB0060E081E00E94BB00512CC7
S11303F0612C712C411451046104710409F03FCF44
S1130400DBCF8DE00E94C800682F6F778DE00E94DB
S1130410BB00C3E00FC08DE00E94C800682F6F7757
S11304208DE00E94BB0086E00E94C8008B7109F435
S113043060CFC3E08C2FDF91CF911F910F91FF907C
S1130440EF90DF90CF90BF90AF909F908F907F9070
S11304506F905F904F903F900895EF92FF920F93AB
S11304601F93CF93DF9300D000D0CDB7DEB7182F02
S11304707B0167E08DE00E94BB00F70110838E01D1
S11304800F5F1F4F970141E0B7018CE00E94FE000F
S1130490813059F449815A816B817C814031510505
S11304A06105710519F083E001C083E00F900F909E
S11304B00F900F90DF91CF911F910F91FF90EF90CC
S11304C00895289A82E48A95F1F700C0289882E476
S11304D08A95F1F700C00895CF93DF93EC016EE2A3
S11304E071E00E940C03892B11F4299A09C063E37B
S11304F071E0CE010E940C03892B11F485B185B9FA
S1130500DF91CF910895CF93C82F83E391E00E94A8
S11305106C02CBB90E946102CF910895CF93C82F8A
S11305208EE291E00E946C02CBB90E946102CF91ED
S11305300895CF93DF93EC018881882361F021969D
S11305400E948E028FE891E00197F1F700C000004D
S113055089918111F5CFDF91CF9108951BB88FEF69
S11305608AB985B18C7F85B984B1836084B92FE35E
S11305708DE093E0215080409040E1F700C00000FE
S113058080E30E9483022FE38DE093E021508040BA
S11305909040E1F700C0000088E00E9483022FE34E
S11305A08DE093E0215080409040E1F700C00000CE
S11305B081E00E9483022FE38DE093E0215080408C
S11305C09040E1F700C000008CE00E9483022FE31A
S11305D08DE093E0215080409040E1F700C000009E
S11305E088E30E9483022FE38DE093E02150804052
S11305F09040E1F700C000000895409A389A84B111
S11306008C6284B98CB581658CBD08958EBD0DB4A2
S113061007FEFDCF8EB50895FB01DC018D9101909D
S111062080190110D9F3990B0895F894FFCFB7
S113062E4D49464152452052433532327632004DC1
S113063E49464152452052433532327631004E6F8F
S113064E2072656164657220666F756E6400646104
S113065E746100696E737472756374696F6E0000F1
S9030000FC
